:1000000075C09BC08CC299C098C097C096C095C05F
:1000100094C093C092C091C033C18FC08EC0000005
:1000200000000000000000000000000023456C9864
:10003000C9FF040714233764A0FFFFFFFFFFFFFF82
:10004000FFFFFFFFFF000000000000000000234052
:100050005F7AB4FFFFFFFFFFFF00140008140008E1
:100060000E140004080E14000305080E1400040802
:100070000A0E1114000305080A0E101400030508E7
:100080000A0E1012140008000E00080E0004080EDC
:10009000000305080E0004080E1100080E1100F3FD
:1000A000F404080E10121400080A0C0E0F1012149B
:1000B00000080EED14000203040500041400040EF1
:1000C0001400040810140004080F1114000305089C
:1000D0000A0E0004080A0E00EEEDECEB140E080404
:1000E0000004080E00EBECEDEEF3F41411241FBE37
:1000F000CFE5D2E0DEBFCDBF20E0A0E6B0E001C09A
:100100001D92AB37B207E1F7ECE7F0E085E58087B9
:1001100081E0838314821282868311828BE082873E
:1001200088E58387E1E6F0E08DEF87838EEF8583B6
:10013000712C55245A94A5D019C262CF1BBC19BC8E
:1001400018BC089520ED37E0019720F0F9013197B0
:10015000F1F7FACF089588EE93E0F4CF369A369906
:10016000FECF95B18091600089270895CF93C72D68
:1001700081E0870D8F73782E662D90E0E9D16FEFC7
:100180008C2F90E0CF91E4C1FF920F931F93CF93F8
:10019000DF93F82E0DE710E0CEE7D0E0F11005C0B8
:1001A000CE01CED1F801808304C0F8016081CE0178
:1001B000CFD121970F5F1F4FC337D10579F7DF915B
:1001C000CF911F910F91FF900895D0DF81E0DCCF98
:1001D000811101C0B3CF815090E0FC01E25EFF4F7E
:1001E000E491EBBDFC01EE5CFF4FE491E9BDFC0145
:1001F000EA5BFF4F849188BD08950F931F93CF93BF
:10020000C82F8B01CC2359F085E0E2DFC8019ADFCB
:1002100095DFC80197DFC80195DFC150F3CFCF91BB
:100220001F910F910895CF93DF93D82F64E170E071
:100230008AE0E3DF84EF91E085DF8D2F64E674D1FF
:10024000CAE06C2F71D1892F68EC70E0D6DF83DFB4
:100250008D2F6C2F69D1D92F67D1892F68EC70E071
:10026000CCDF79DF68EC70E08D2FC7DF74DF64E1ED
:1002700070E08AE0C2DF84EF91E0DF91CF9162CF3E
:10028000189510927B0087E790E05AD1853519F0D8
:10029000612C9BDF11C0712C872D90E051D1682E0D
:1002A0008F3F19F080E070DF07C0872D91E0970D38
:1002B000792E803488F3F6CF90918600D0917F001C
:1002C00010918000C0917D00CC2319F010E0D0E0A7
:1002D0009AE19F5F80E040E050E06AE570E099239A
:1002E00079F09B012F5F3F4FF9013197E491EE23A5
:1002F00019F0822F861BF6CF9150AB01B901EFCFD9
:10030000982F6D2F70E0A82FB0E0E92FF0E01123B7
:1003100021F09D012E1B3F0B05C09F01215031098B
:10032000260F371F3197E40FF51F049125593F4FD2
:10033000F9010083915049F78D0F80938800DD23E8
:1003400071F0112329F0282F30E02150310902C02B
:1003500020E030E0F901E559FF4F91E0908397E00C
:10036000980F292F2150E22FE81BF0E0EB51FF4FAF
:10037000E491A22FB0E0A559BF4FEC932813F2CF20
:10038000E92FF0E0E659FF4F21E040916B0030810A
:10039000431320E0921B90938900262D253FE8F51A
:1003A000352D3330B0F490918A009F3F29F480912D
:1003B0007B0080938A0006C091E0960D692E981705
:1003C00008F0612C80918A008F5F8F7180938A0082
:1003D00024C020917B0020938A003630C0F4209105
:1003E0008200222311F0CC2339F091E0960D692E82
:1003F000981798F0612C11C0262D6816D9F3662045
:1004000019F02150622E09C09150692E06C0C11109
:10041000F1CF80917E00882369F3512C8FEF8DBD41
:1004200080E68CBDAA9AAA9A8FE384BB8BE187BB36
:1004300080EE88BB81E083BF91EA9ABD80BF8BB715
:1004400080628BBF8AB785608ABF85B7806285BFAF
:1004500078948CE287B986EC86B93699FECF8FEF17
:10046000809360008CE291E06DDE78DEDCDEFACF16
:10047000112416B863DE87B3847E87BB80E061E019
:1004800034E0A4E040E25EE496B39A27999B03C06F
:10049000511003C03CC0911108C025E0251508F09B
:1004A00038C0811136C060E039E0252D71E0273079
:1004B00008F070E0270F522E263019F4FA01319718
:1004C000F1F7611108C0811105C081E0911103C0ED
:1004D00080E001C081E0999895B7977E906195BFC3
:1004E000A895932F987011F420E401C020E6932F73
:1004F0009770922B91BD95B7946895BF9B7F95BFE0
:1005000078948895F89491B59F7B91BDBDCF91115A
:10051000CCCF8FE58DBF82E08EBF1FBEB2DE5520EF
:1005200011F0189501C0A4DF991B79E004C0991F50
:10053000961708F0961B881F7A95C9F7809508953D
:10054000E199FECF9FBB8EBBE09A99278DB30895AA
:10055000262FE199FECF1CBA9FBB8EBB2DBB0FB6D9
:10056000F894E29AE19A0FBE01960895F894FFCFAD
:00000001FF
